:030000000208A84B
:080003000280038E828F83222C
:08000B0002800BAE82AF8322DC
:08001300028013742D0173003B
:08001B0002801B11730171004A
:08002300028023111601710097
:03002B0002802B25
:10002E00217601730167216521872194018A01CE12
:10003E0021CE21A8020922020B41017D0201BB0241
:10004E000A8A020A90020ACE02086902082F0207E3
:10005E00BA020790020A09214A3098FDC298E59922
:10006E0022117174203099FDC299F59922117DC02B
:10007E00E0740D1173740A1173D0E022C2D51162AF
:10008E0031A8B41B03D3E422B40D05D2D5C3E422A8
:10009E00FA314A40E9CA1173116231A8B41B0280C9
:1000AE00E4B40D03EAC322B40804117380D0B4156E
:1000BE000280F7FB314A40E0CB1173EAC44BC322F6
:1000CE007A007B007C04C2D5116231A8B41B07D321
:1000DE00E4F583F58222B408028003B47F0CBC04DD
:1000EE000280E5117331390C80DEB40D108B838ADA
:1000FE0082BC0407E4F583F582D2D5C322FD314AD2
:10010E0040C6CD120073EDC0E03128D0E02AFAE4EB
:10011E003BFBDCB4C38A828B8322EBC454F0FBEA34
:10012E00C4540F4BFBEAC454F0FA22EAC4540FFA3B
:10013E00EBC454F04AFAEBC4540FFB22C324D05044
:10014E001424F64004240AC32224F9500824FA4049
:10015E00042410C322D322C0E0C4540F24F650024C
:10016E002407243A1173D0E0C0E0540F24F6500255
:10017E002407243A1173D0E022C0E0E5833165E50F
:10018E00823165D0E022C0E0E493A3600AA2E75476
:10019E007F1173400280F1D0E022C0E0C394614031
:1001AE0009941A5005D0E024E022D0E0227800C055
:1001BE00E0E4936008A2E7084003A380F4D0E022B5
:1001CE00C0E0C3309808E599B41B01D3C298D0E0C3
:1001DE0022900DDD1145EF3165EE316531941162DE
:1001EE0031A875F0DFC0F075F001C0F0F5F0901099
:1001FE0000F1905024758204E493B4FE150582E458
:10020E0093B5F00E11717582203194117D75824077
:10021E00E4730583E583B400D8E5F0B43F07900F8F
:10022E00461145A1D4B44D07900F4E114581C4B46B
:10023E005207900F531145A13BB44407900F57112D
:10024E004541A8B45507900F5A1145C149B44E0700
:10025E00900F5D1145E13BB44A07900F6111458146
:10026E0012B44807900F6711458149B44507900FA6
:10027E00731145818AB44307900F781145E117B485
:10028E005A0B74006012900F7C1145E14BB4490873
:10029E00900F6D1145020771017D900E7811457812
:1002AE00107A10760008DAFB1167B41B028072B464
:1002BE003A0679007141800A314A40EC7906714163
:1002CE0080E6742E11737C007160F87160F5837195
:1002DE0060F5827160B40102802D7022E8601471A5
:1002EE0060FA79017141EA120869E43402F9714148
:1002FE00A3D8E97160EC60B07904714180AAE8601E
:10030E00F27160D8FC80ECE860047160D8F3716023
:10031E00EC70E57138900E97114530987A11678020
:10032E00767138900E8F1145806D78007900D9FE68
:10033E00D8FA22E95407232410F907E770020907B7
:10034E0022D3878209878309E5827005E5837001D0
:10035E00C322116731A8B41B06D0E0D0E080C2B42E
:10036E003A0A79057141D0E0D0E041D0314A5006C9
:10037E007907714180DCFA116731A8B41B0280D96C
:10038E00B43A0280DD314A50067907714180E8CADD
:10039E00C44AFA2CFCEA22EEC0E0EFC0E0900E9EBA
:1003AE00114579107EA77F0E910E7EAD7F0E910EB8
:1003BE007EB27F0E910E7A05714F4009DAFA900ED9
:1003CE00EE11458025900EBD114579167EC17F0E2A
:1003DE0091007ED27F0E91007EDA7F0E91007EE03C
:1003EE007F0E91007EE57F0E9100D0E0FFD0E0FE03
:1003FE00017D714F50091171120ACE11061145225D
:10040E00714F80F2900E1F114511063187900DED40
:10041E00114511CE20D5065002E112110E117D901C
:10042E000EFC11451106E4F5D0F5F0F8F9FAFBFCD7
:10043E00FDFEFF758108C0E0C0E0737A10117B11DC
:10044E00063187743A111E7B101106E493A33165B1
:10045E001171DBF7116F7B101106E493A3547FB477
:10046E007F01E424E04001E424201173DBEC117DD4
:10047E00D1CE110E31CE4002DAC5017D900E611142
:10048E004511CE110E117D3187743A111E7428114B
:10049E0073110EE4933165900E3A1145118A20D5F1
:1004AE0010400E1106120869117D1106A3110E815E
:1004BE0095900E6D0145900E29114578151171D844
:1004CE00FC1145758310F1904002017D116F75820C
:1004DE0020319475822031BB7421C398F874201199
:1004EE0073D8FC7582003187780674201173D8FC9E
:1004FE00758204E493AA83B4FE05900F348018B479
:10050E00FD05900F3B8010B42305900F388008B482
:10051E00F90280EE900F4211458A83117D74FFB56A
:10052E00830281D80583E583B4009B81D8117B7A41
:10053E00FF90100015830583E583B400028021F13E
:10054E0090501D758204E4934403F460E9116F0A20
:10055E0074412A111E11267582203194117DA144F9
:10056E00BAFF05900DF60145900DE8114574411145
:10057E0073111674412A1173900DED11451162B469
:10058E001B02017DFB741FC39AEB400231A811734D
:10059E00FB117DEBC3944140CFFBEAC39B40C90BDB
:1005AE0090100015830583E583B400028017F19047
:1005BE005013758204E4934403F460E9DBE7117D84
:1005CE00758240813422900F1C11457C3F900F495B
:1005DE00D13E7C4DD13E7C52D13E7C44D13E7C55A9
:1005EE00D13E7C4ED13E7C4AD13E7C48D13E7C49A8
:1005FE00D13E7C45D13E7C43D13E740060047C5A92
:10060E00D13E900F2A1145901000F1905020758226
:10061E0004E493B4FE11116F0582E4931173112655
:10062E007582203194117D0583E583B400DC017D54
:10063E00116FEC117311261145017DD1E0900F065B
:10064E001145EB3165EA31651145ED3165EC3165EA
:10065E00117D8D838C82A3AC82AD83900E151145D6
:10066E001167B41B02E110117D8A828B83ECC39556
:10067E0082FAED95837009EA603254F070028002BE
:10068E007A10743A1173EA31653187E58325822A2F
:10069E00FBE43165E49331652BFBA3DAF7EBF4044D
:1006AE003165117DD1CE31CE50C38056743A11735F
:1006BE00E431653165316504316574FF3165017B67
:1006CE00E8C0E0780CE58C04000070FBD8F7D0E0B1
:1006DE00F822117B900E43114511CE402120D51EDC
:1006EE00C083C082117D900E4D114511CEAD83ACED
:1006FE0082D0E0FAD0E0FB400520D502017DD0E0AB
:10070E00D0E0117D900DD50145D1E0900E571145E9
:10071E00116231A8B459EB117B8B838A82E41208E3
:10072E0069EDB58305ECB5820122A380F0900E0C25
:10073E00114511CE40CE20D5CB110E017B117B90F1
:10074E000F7C1145742C111E900E571145116231FC
:10075E00A8B459AE117B1207BA900F815003900FB7
:10076E00880145117D7800117DE83165743A117369
:10077E001171E6316508E8540F70F5117DB800E986
:10078E00017D758200E493B4A517A3E493B4E5113B
:10079E00A3E493B4E00BA3E493B4A505758200D350
:1007AE002274FFB58302C322058380D6740060389D
:1007BE00908000E493F4700DA37400B582F574007C
:1007CE00B583F0C322908000E4936006E412082FF4
:1007DE004016A37400B582F07400B583EB908000D0
:1007EE007CE87D04DC04DD02D3227420A2AF92D11A
:1007FE00C2AFF0F07B147AE5DAFEDBFA74A0F07A81
:10080E0005DAFEE493A2D192AFF470D8A37400B5CA
:10081E0083EA7400B582E574FF908000F0E4F0C3C3
:10082E0022F5F0EAC0E0EBC0E07A197440A2AF9274
:10083E00D1C2AFF0E5F0F07B13DBFE74C0F07B05A8
:10084E00DBFEE493A2D192AFC395F06003DADCD362
:10085E00E4F0D0E0FBD0E0FAE5F022C0E0C0F0F525
:10086E00F07400601BE583B4FF02800B5012B4805D
:10087E0002800450028009E5F0112FD0F0D0E02262
:10088E00E5F0F0E493C395F06009E0C395F06003E2
:10089E00D38001C3D0F0D0E02232E4F5A8F5B875CC
:1008AE00D00011A711A7F4F580F590F5A0F5B0755D
:1008BE00813079C87AF9DAFED9FA7400601374B50A
:1008CE00600F78FAA2B579C8D9FE4005D8F612079E
:1008DE00BA75F0F911F5312275F0FD11F512007DA2
:1008EE007E007F800201DF90100012079050247569
:1008FE008204E493B5F015C0F0C0837416C0E074A2
:10090E0009C0E0758240E473D083D0F00583E5839F
:10091E00B400D72274007014E57B637A556379CCEA
:10092E0063781DB57A08B57905B5780221E8758723
:10093E0080759842758911E4F588F58AF58CF58BEA
:10094E00F58D78C8791E30B0E5D9FBD8F720B0FD0B
:10095E0020B0FA20B0F720B0F420B0F130B0FDD2C4
:10096E008E208FCA20B0FA208FC430B0FA208FBEEE
:10097E0020B0FAD28C208FB630B0FAC28EC28C2044
:10098E008FACE58B33F5F0E58D3340A2A2F7340042
:10099E00F404609AF58D758BFF758921D29CD28EE9
:1009AE00E58DF404F978FFD8FED9FA309811C29883
:1009BE00E599547F24F660072405600302093CE59F
:1009CE008A33F8E58C33F940F3E833F5F0E933A2D6
:1009DE00F7340060E7F404B58DE2F57BF57AF5792E
:1009EE00F578637A556379CC63781DF58DF58B7543
:1009FE008921758780759852D28E22309806120002
:100A0E0067B41B51120067B41B4B517720980374C7
:100A1E001B22120067B45B4451773098DE120067D8
:100A2E00B44103740B22B44203740A22B443037418
:100A3E001522B44403740822B435028007B436027A
:100A4E0080028018C0E0517730980B120067B47E98
:100A5E0009D0E024E422D0E080A1D0E05177309894
:100A6E009A120067B41BF580A1EAC0E07A14E58CF7
:100A7E002098050470FADAF6D0E0FA22C0F0C0E051
:100A8E008013C0F0C0E030E70C742D120073D0E07C
:100A9E00C0E0F4240175F06484D2D56007C2D52479
:100AAE0030120073E5F075F00A8430D5026005242B
:100ABE0030120073E5F02430120073D0E0D0F02233
:100ACE00C0E0E8C0E0C2D5AA82AB837C107D27715E
:100ADE002C60072430120073D2D57CE87D03712C74
:100AEE00700330D5072430120073D2D57C647D009C
:100AFE00712C700330D5072430120073D2D5EAABB7
:100B0E00F075F00A84700330D5052430120073E5B9
:100B1E00F08BF02430120073D0E0F8D0E022780091
:100B2E0008C3EA9CFAEB9DFB50F618EA2CFAEB3D53
:100B3E00FBE822C0E0E8C0E0E9C0E0ECC0E0D2D1C2
:100B4E00D2D5E493A3602520E72E547FB40D07126F
:100B5E00007DD2D180ECB41F04C2D580E5B40E0561
:100B6E0012007D8007C2D112007380D6D0E0FCD077
:100B7E00E0F9D0E0F8D0E022547FF820D103120043
:100B8E0071C2D1C082C083900BFB7C00E86007F974
:100B9E0071EA70FCD9FA71EA603CB40F1271EA0482
:100BAE0083801E68667767796278766B716A7A04DD
:100BBE0083800E657461726E69736F6C756D70648F
:100BCE0063A2D592E5D2D5B81402C2E5B80C02C222
:100BDE00E512007380C0D083D0826150E493BC00D4
:100BEE00057CFF540F227C00A3C4540F228290E890
:100BFE002386054CF844B3B0B1485FF0117FA015C1
:100C0E007F1C2ED1405A50F103BFBA0C2F96018D86
:100C1E003F95380D6F5F1207710E562F483B625885
:100C2E00201F7670322440B840E1618F01340BCA28
:100C3E0089D3C0A3B9588004F80285602591F0923B
:100C4E00731F107F12549310444807D126564FD06D
:100C5E00F66472E0B83BD5F0164F56306F48025F1F
:100C6E00A8201F017630D5602541A42C60056F01A8
:100C7E003F261F30078E1DF06399F042B8201F23C8
:100C8E0030027AD1602FF0F6058F931A5028F08239
:100C9E00046FA30D3F1F514023013E0543017A010E
:100CAE00176493302A088C243099B0F319602541CB
:100CBE0035098ECB191230051F311D04144F7612D3
:100CCE0004AB279056012FA8D5F0AA26205F1CF062
:100CDE00F361FE0141730127C1C0848FD601877075
:100CEE00564F19701FA8D99076021743FE01C18482
:100CFE000B157F028B14308F63396F19F011C910E9
:100D0E006D023F91097A41D0BA0C1D395F07F2117D
:100D1E001720416B3509F775120BA7CC48023F64BB
:100D2E0012A00C27E39FC014777011407121C06888
:100D3E002541F0627FD1D021E16258B0F3051F73D7
:100D4E003077B16F19E01943E0582FF6A414D02371
:100D5E0003FE31F5143099F8033F642251602541AA
:100D6E002FE30156279309FE11FE79BA607542EA08
:100D7E006258A0E51F534FD1C0A3094253F7120486
:100D8E00621B30F505F7690C351B70822F2F144F3F
:100D9E0051C064250057656C636F6D658094322C6D
:100DAE002062791FF81FFE0D0E20205365659432C8
:100DBE002E444F432C94322E455155A494322E4836
:100DCE004452B4D58D2E0E201F9E1FA0210D0E94C1
:100DDE0032204C6F633A00203EA086CA822800293A
:100DEE002C958C80C83A20001F9782C373C7A683A8
:100DFE002CBA204A554D508086A172820D0E0D0DD3
:100E0E001F8783813A20001FE4FB206B65793A200F
:100E1E00000D0D1F888083812028000D0D1F821F5D
:100E2E00FD001F8120202020201FC90E29201F8792
:100E3E001FB23A200046697273741F813A20004C2B
:100E4E006173741F813A2020001FB9A1207375723F
:100E5E00653F000D0D416464726573733E20002082
:100E6E00201F9CC12C8E81F70D0E0D0D1F9F206132
:100E7E0073636969F9961F9884892C958C80A00DEF
:100E8E000E0D1F8AA065640D0E0D1F8AC1640D0E16
:100E9E0053756D6D6172793A0E20C67391640E2092
:100EAE008B91640E208B207772697474656E0E1FA1
:100EBE009B3A0E208B20756E61626C658020777276
:100ECE006974650E2020626164F5730E20859F960D
:100EDE00C60E2085849D0E2085206E6F6E849D0E1D
:100EEE001F979B2064657465637465640D0E0D8693
:100EFE006E696E67823A0D0E0D0D53656E64696EE6
:100F0E00671F988489AC20200020802020000D0DC2
:100F1E005374616E646172641F9E730E1FDA1FF448
:100F2E0065641F9E730E1F9A9E001F82001F8F1FE7
:100F3E00E21FAA003F3F3F001FD7001F8ED7D100F0
:100F4E001FD18273001F8682001F8A001F93001F0D
:100F5E008781001F88808381001F84DB9A83001F96
:100F6E0084DBC083001F9C9A92001FED83001FCB71
:0F0F7E009990001F9990CB640D0E1F859B0D0E4F
:00000001FF
